:020000040000FA
:100000008316C73081008E100E14FF23900000303D
:100010009500831285010730990083160F30850003
:1000200073309F008312A8018512051205158515EE
:100030002C102E102F1026143F30AA009E232B08C0
:10004000A600AB01AA0127147F30AA009E232B082B
:10005000A700AB01AA017C206430250203183128D7
:100060002F147C209B302502031C37282E14732369
:10007000C322D5227323562056204A2056206B20B7
:100080004A2056204A206B204A204A204A205620E7
:100090007923752805160230A0001930A100FB2035
:1000A000A10B4F28A00B4D2805126128051606301C
:1000B000A0001930A100FB20A10B5B28A00B592840
:1000C00005120230A0001930A1000221A10B652801
:1000D000A00B632808000430A0001930A100022101
:1000E000A10B6F28A00B6D28080087280130802005
:1000F000A4000310A40C080005308020A50008000F
:100100009F0068239F149F1883281E0808007C20E6
:1001100064302502031C092968237C2064302502F1
:10012000031C092968237C209B3025020318182909
:1001300068237C209B302502031818296823851D1D
:10014000A428051DC22887287620A3018516051638
:100150000230A0002408A100A01CF320FB20A10B6A
:10016000AC28A00BAA28051285120230A000240892
:10017000A1000221F320A10BB928A00BB728A318D6
:10018000C22887287620A3012E18E2288516051696
:100190000630A0002408A100201DEB20FB20A10BAD
:1001A000CC28A00BCA28051285120230A000240812
:1001B000A1000221EB20A10BD928A00BD7282318DE
:1001C000A428872885160516A301EB20051DE52820
:1001D00005128512D5288519F22868238519F22879
:1001E0000130A30008000519FA2868230519FA2828
:1001F0000230A30008007D30A200FE28FF28A20BD9
:10020000FD2808007630A20005290629A20B042942
:1002100008000A30B30073237C20643025020318E1
:10022000522AB30B0B297F23E722C32273232729EA
:100230000A30B30073237C209B302502031C592A0B
:10024000B30B1A297F23E722D52273233A293D23B2
:100250003E30A8000030AA000830A9000830AD00E8
:100260007C2064302502031C162A851D4D29051D9E
:100270008F292E2953233E30A8004030AA00083091
:10028000A9000830AD007C209B3025020318342AD9
:10029000851D5D29051D9A2941296D21AD0B532925
:1002A0007923051214297C2064302502031C162AA8
:1002B000851D4D29051D8F29C9296D21AD0B632988
:1002C0007923051223297C209B3025020318342A28
:1002D000851D5D29051D9A29D22976202B1403102E
:1002E000AB0DA9032B10DB21A30105160230A000E2
:1002F0002408A100A01CF320FB20A10B7A29A00B4D
:10030000782905120230A0002408A100F320022160
:10031000A10B8629A00B8429A318A5290800A521D3
:100320007C2064302502031C162A851D4D29051DDD
:100330008F29C929A5217C209B3025020318342A46
:10034000851D5D29051D9A29D22976202B100310C1
:10035000AB0DA9032B14DB210516A3010630A00069
:100360002408A100201DEB20FB20A10BB229A00B2B
:10037000B02905120230A0002408A100EB200221C0
:10038000A10BBE29A00BBC2923186D290830AD0094
:1003900008002610E9210830AD00F021E921E9210B
:1003A0004A202E292710E9210830AD000322E92137
:1003B000E9214A204129A90BE129A723A80BE42917
:1003C000142B0310AB0DE829AA0A0830A900AB01D1
:1003D00008002B140310AB0DA9032B14DB2108001C
:1003E0000A30A0002408A10002217C2064302502EC
:1003F000031C162A851D4D29051D8F29A10BF429E3
:10040000A00BF22908000A30A0002408A100022154
:100410007C209B3025020318342A851D5D29051D8B
:100420009A29A10B072AA00B052A08007923C322C9
:100430002618FE2A2B100310AB0DA9032B10A90BB5
:10044000222A282A0310AB0DA903AB0DA90B222ADF
:10045000A7232608AB003F30AA00A723A8012C142D
:1004600060222A232C1087287923D5222718FE2AD8
:100470002B100310AB0DA9032B10A90B402A462A01
:100480000310AB0DA903AB0DA90B402AA723270826
:10049000AB007F30AA00A723A8012C1465222A23D1
:1004A0002C1087282618FE2A60222F1CF22A8B2364
:1004B000542A2718FE2A65222F1CF22A8B235B2A36
:1004C0006D230030AA006A2208006D234030AA0084
:1004D0006A2208009E230830A900AB1F702A762AE2
:1004E000A9030310AB0DAB1F822A7E2AA9030310B8
:1004F000AB0DAB1F802A7C2AB822832A9C22832A38
:100500008A22832A0800A90B872AAA0A6A2A0310CA
:10051000AB0D6D2A76202C188E2A85160516023012
:10052000A0002408A100FB20ED22A10B932AA00B20
:10053000912A05128512AD2A76202C18A02A85163C
:1005400005160630A0002408A100FB20ED22A10B17
:10055000A52AA00BA32A051285120230A0002408A8
:10056000A1000221ED22A10BB12AA00BAF2A0800A5
:100570000430A0002408A100FB20ED22A10BBC2A1E
:10058000A00BBA2A08007C2064302502031CC32A71
:100590006D237C2064302502031CC32A6D237C203C
:1005A00064302502031CC32A08007C209B302502EE
:1005B0000318D52A6D237C209B3025020318D52AE9
:1005C0006D237C209B3025020318D52A0800562075
:1005D0004A204A204A2056200800851DF22A051D7F
:1005E000F22A08007323A001A101A20105128512BD
:1005F000851DF82A051DFA2A2C10872879235620F4
:100600004A206B205620562056206B206B206B20F2
:1006100056204A204A206B204A2056206B20562024
:100620006B204A2056208728732356204A206B20AF
:100630005620562056206B206B206B204A205620D7
:100640004A206B205620562056206B2056205620DC
:100650006B20872873236B205620562056206B2052
:1006600056204A2056206B206B206B204A204A20BF
:10067000562056204A204A2008004030A80000306A
:10068000AA002A0883169B001C1555309D00AA302D
:100690009D009C149C184A2B9B0A8312A80B452B87
:1006A00026141C1108004030A8004030AA00831610
:1006B0009B001C1555309D00AA309D009C149C1871
:1006C0005F2B9B0A8312A80B5A2B27141C110800BE
:1006D0000F30B000B00B6A2B0800B530B1006823B2
:1006E000B10B6F2B08000A30B2006D23B20B752BD3
:1006F00008001E30B2006D23B20B7B2B0800643063
:10070000B2006D23B20B812B0800C830B2006D23FC
:10071000B20B872B08001730B200ED226430B10015
:100720006430B000932B942B952B962B972BB00B0A
:10073000922BB10B902BB20B8D2B080083122A0841
:1007400083169B001C141A088312AB000800831246
:100750002A0883169B0083122B0883169A001C1507
:100760008B1355309D00AA309D009C149C18B62B0D
:0A0770001C118B171C1183120800E6
:02400E00843FED
:00000001FF
